:0200000480007A
:100000006F008004732F2034930F80006308FF0378
:10001000930F90006304FF03930FB0006300FF038E
:10002000130F000063040F0067000F00732F2034CC
:1000300063540F006F00400093E19153171F0000BD
:1000400023223FFC6FF09FFF93000000130100008C
:10005000930100001302000093020000130300004C
:100060009303000013040000930400001305000034
:10007000930500001306000093060000130700001C
:100080009307000013080000930800001309000004
:1000900093090000130A0000930A0000130B0000EC
:1000A000930B0000130C0000930C0000130D0000D4
:1000B000930D0000130E0000930E0000130F0000BC
:1000C000930F0000732540F16310050097020000B4
:1000D000938202017390523073500018970200000F
:1000E0009382020273905230B70200809382F2FF33
:1000F0007390023B9302F0017390023A73504030C8
:100100009702000093824201739052307350203066
:100110007350303093010000970200009382C2EECA
:1001200073905230130510001315F501634C050050
:100130000F00F00F930110009308D0051305000085
:100140007300000093020000638A02007390521053
:10015000B7B2000093829210739022307350003037
:10016000970200009382420173901234732540F18C
:1001700073002030930000001387000093030000F9
:1001800093012000631C7726930010001387100052
:100190009303200093013000631277269300300010
:1001A000138770009303A000930140006318772425
:1001B0009300000013870080930300809301500098
:1001C000631E7722B700008013870000B70300800A
:1001D0009301600063147722B700008013870080CA
:1001E000B703008093830380930170006318772026
:1001F000930000001387F07F9303F07F930180004A
:10020000631E771EB70000809380F0FF1387000005
:10021000B70300809383F3FF930190006310771E70
:10022000B70000809380F0FF1387F07FB703008052
:100230009383E37F9301A0006312771CB7000080D3
:100240001387F07FB70300809383F37F9301B0009F
:100250006316771AB70000809380F0FF1387008041
:10026000B7F3FF7F9383F37F9301C0006318771880
:10027000930000001387F0FF9303F0FF9301D00079
:10028000631E77169300F0FF13871000930300009E
:100290009301E000631477169300F0FF1387F0FFDB
:1002A0009303E0FF9301F000631A7714B700008016
:1002B0009380F0FF13871000B703008093010001C3
:1002C000631E77129300D0009380B00093038001E7
:1002D0009301100163947012130200009300D00088
:1002E0001387B000130307001302120093022000CB
:1002F000E31652FE930380019301200163107310F3
:10030000130200009300D0001387A0001300000028
:10031000130307001302120093022000E31452FE9D
:100320009303700193013001631A730C13020000F0
:100330009300D0001387900013000000130000000A
:10034000130307001302120093022000E31252FE6F
:1003500093036001930140016312730A13020000CA
:100360009300D0001387B000130212009302200004
:10037000E31852FE93038001930150016310770844
:10038000130200009300D000130000001387A000A8
:100390001302120093022000E31652FE9303700131
:1003A00093016001631C7704130200009300D000E6
:1003B00013000000130000001387900013021200C6
:1003C00093022000E31452FE930360019301700135
:1003D00063167702930000029303000293018001E9
:1003E000639E7000930010021380200393030000AB
:1003F0009301900163147000631030020F00F00F3E
:10040000638001009391110093E111009308D005DE
:1004100013850100730000000F00F00F930110001E
:100420009308D0051305000073000000731000C08E
:0C043000000000000000000000000000C0
:1010000000000000000000000000000000000000E0
:1010100000000000000000000000000000000000D0
:1010200000000000000000000000000000000000C0
:1010300000000000000000000000000000000000B0
:081040000000000000000000A8
:040000058000000077
:00000001FF
